:020000040000FA
:10000000492882070B340934063407340C3403348E
:100010000D340A3405340E34033409340A340D34F3
:1000200005340E340C348207AB349534EC34BD34D3
:10003000553477347A343934DD34663479346D3478
:10004000AC343C34E734BB3459349E34DB34CD34E7
:10005000A7349334DE34B5346C349734E934ED345A
:1000600033348207013405340F340A340134033445
:100070000A34053405340F340F340A34013405349E
:1000800001340A340F34013401340A3405340534A0
:100090000A3483168501860183128F019001910134
:1000A00085018601802080202B3093000F080120DD
:1000B00085008F0A0F08113C03198F0110081320C7
:1000C0008600900A10081D3C031990011108312088
:1000D00092008020920B6928910A1108173C03199D
:1000E0009101930B562805309300850186018020ED
:1000F0000F308500FF3086008020930B7528502834
:1001000002308C00F3308D0000308E0000008E0B2A
:0C01100086288D0B84288C0B82280800A8
:02400E00FA3F77
:00000001FF
